:1000000014C600007EC600000C94412D7AC6000084
:100010000C941B2D76C6000074C6000072C600004A
:1000200070C600006EC600000C94252C6AC6000045
:100030000C94002C66C6000064C6000062C6000076
:1000400060C600005EC600005CC600005AC6000024
:1000500058C600000C94DA2B54C6000052C60000AB
:1000600050C600004EC600004CC600004AC6000044
:1000700048C6000046C6000044C6000042C6000054
:1000800040C600003EC600003CC600003AC6000064
:1000900038C6000036C6000034C6000032C6000074
:1000A00030C600002EC600002CC600000631FF0935
:1000B00074A1010975150026FF00952075088102BD
:1000C0000976150026FF00952075089102C00501EC
:1000D0000902A1010901A1008501050919012908E9
:1000E00015002501950875018102050109300931C6
:1000F0001581257F95027508810609381581257FB0
:10010000950175088106050C0A38021581257F9531
:100110000175088106C0C005010980A1018502168C
:1001200001002637001A81002AB700751095018159
:1001300000C0050C0901A1018503160100269C02DF
:100140001A01002A9C02751095018100C005010961
:1001500006A101050719E029E71500250195087595
:10016000018102050819012905950575019102957E
:1001700001750391010507190029F715002501955F
:10018000F875018102C05220006973723A2530343B
:100190005820007725303258200072253032582000
:1001A000000A5B434C525D2000214353325F4530CF
:1001B0005F4630210A00214353325F46302120251B
:1001C0003032580A00214353325F4530210A002162
:1001D0004353325F494E4954210A00214353335F50
:1001E0004630210A00214353335F5245414459218F
:1001F0000A00214353335F5245534554210A0045B9
:100200002575200050257520004D5B783A25642027
:10021000793A256420763A256420683A256420627C
:100220003A253032585D0A004C257520000A4D6F82
:100230007573653A2025730A000A4445463A200042
:100240000A4558503A20000A494E543A20000A4CB8
:100250004F473A20000A4C4D533A20005325752051
:10026000000A49443A25303458282573257329203B
:10027000000A556E6B6E6F776E2049443A205265C6
:10028000706F727420746F20544D4B20004F4B20C0
:10029000004E4720004F4B20004E47200A54656C0B
:1002A00065766964656F3A20000A353537365F43F5
:1002B000533832683A2000522575200057257520A2
:1002C00000572575200057257520005825752000FA
:1002D000412575200049257520005B4348475D2076
:1002E000000A2575205052543A253032582049537F
:1002F000523A2530345820000A2575204552523A8A
:1003000025303258204953523A25303458200000C5
:100310007B46010203763A687F6577482B353B6957
:1003200078796439141E3C6A7A1D16041A1F3D6BD5
:10033000061B070821203E6C2C19091715223F6D5A
:1003400011050B0A1C23406E7E100D182425416FE9
:10035000360E0C122726427037380F33132D437197
:100360007534322F2E44727C7D28303174457351A0
:10037000504A524D492A5466594F5C5F4C4B4E626D
:10038000635A5D5E60295367585B5657614755480D
:1003900042403E3C3A3B456843413F3D2B357E69F8
:1003A0007A790078141E7B6A7C1D16041A1F7F6BF5
:1003B000061B07082120656C2C19091715224A6DA8
:1003C00011050B0A1C234C6E49100D182425516F82
:1003D000360E0C1227264F7037380F33132D5271FB
:1003E0007534502F2E4E72397D28304D314B735459
:1003F00064586776012A773259745C5F660203623B
:10040000635A5D5E60295344575B56556147468089
:10041000291E1F20212223242526272D2E2A2B1496
:100420001A0815171C180C12132F302878041607F9
:10043000090A0B0D0E0F33343579311D1B061905D2
:1004400011103637387D557A2C393A3B3C3D3E3FCA
:100450004041424353475F6061565C5D5E57595A65
:100460005B62634648644445677B7F6503010252D3
:1004700050514F68696A6B6C6D6E6F707172580085
:10048000494C754A4D734B4E767C777E7466545357
:100490005B25303258202530325820253032585DC7
:1004A000200025583A253031366225730A000A208B
:1004B00020303132333435363738394142434445C0
:1004C000460A004C45443A20253032580A000A4C6E
:1004D0006F6F702073746172742E0A000A55534254
:1004E00020636F6E666967757265642E0A000A5430
:1004F0004D4B3A3163353238612F4C5546413A64A1
:1005000036613764660A0009025400030100A03214
:100510000904000001030101000921110100012269
:1005200039000705810320000109040100010301CE
:100530000200092111010001227F00070582030842
:10054000000109040200010300000009211101005B
:10055000012222000705830320000112011001007F
:10056000000008EDFEEE1B01020102000134034908
:100570000042004D0020005000430020006B006549
:1005800000790062006F0061007200640020006367
:10059000006F006E007600650072007400650072E6
:1005A000000000080354004D004B00000004030944
:1005B0000473797374656D3A20253034580A0063EA
:1005C0006F6E73756D65723A20253034580A003F9E
:1005D000004D3E2000433E20000A00257500363ABB
:1005E00020776865656C5F74696D655F746F5F6DBA
:1005F00061783A20000A00257500353A2077686551
:10060000656C5F6D61785F73706565643A20000AA0
:1006100000257500343A2074696D655F746F5F6DF5
:1006200061783A20000A00257500333A206D617820
:100630005F73706565643A20000A00257500323AE0
:1006400020696E74657276616C286D73293A20009A
:100650000A00257500313A2064656C6179282A31D9
:10066000306D73293A20000A092D2056616C75659A
:1006700073202D0A004D3E004D25643E20003F00B2
:100680007365742064656661756C740A00433E206E
:10069000000A002530325820006B6579626F617264
:1006A000643A2000290A002575002F002575005D99
:1006B0002800256400200025640020002564002017
:1006C000002564007C0025303258006D6F7573651D
:1006D0006B6579205B62746E7C7820792076206867
:1006E0005D287265702F61636C293A205B000A09EE
:1006F0002D204D61676963202D0A643A09646562A3
:1007000075670A783A096465627567206D6174726D
:1007100069780A6B3A096465627567206B6579626E
:100720006F6172640A6D3A096465627567206D6F66
:100730007573650A763A0976657273696F6E0A7326
:100740003A097374617475730A633A09636F6E735F
:100750006F6C65206D6F64650A302D343A096C61E9
:10076000796572302D34284631302D4634290A50AF
:100770006175733A09626F6F746C6F616465720AB8
:100780006E3A094E4B524F0A000A092D20436F6EF4
:10079000736F6C65202D0A4553432F713A097175AB
:1007A00069740A6D3A096D6F7573656B65790A0036
:1007B0003F004E4B524F3A206F66660A004E4B5236
:1007C0004F3A206F6E0A0074696D65725F726561E1
:1007D00064333228293A202530346C580A006B657E
:1007E00079626F6172645F6E6B726F3A2025580A8E
:1007F000006B6579626F6172645F69646C653A2051
:1008000025580A006B6579626F6172645F70726F60
:10081000746F636F6C3A2025580A00686F73745FB9
:100820006B6579626F6172645F6C65647328293AE5
:100830002025580A000A092D20537461747573200D
:100840002D0A004743433A20372E332E302041569D
:10085000522D4C4942433A20322E302E3020415600
:10086000525F415243483A20617672350A004F5038
:1008700054494F4E533A204C554641204D4F555305
:10088000454B45592045585452414B455920434FFB
:100890004E534F4C4520434F4D4D414E44204E4BFF
:1008A000524F204B45594D41505F53454354494F9A
:1008B0004E20424F4F544C4F414445525F53495A8A
:1008C000450A004255494C443A203163353238617B
:1008D000202832313A35393A3030204A756C2020A0
:1008E000352032303233290A005649443A203078D4
:1008F0004645454428544D4B29205049443A203020
:1009000078314245452849424D205043206B657956
:10091000626F61726420636F6E76657274657229AE
:10092000205645523A203078303230310A00444562
:1009300053433A204445534352495054494F4E0A79
:10094000000A092D2056657273696F6E202D0A000A
:100950000A6D6F7573653A206F66660A000A6D6FDF
:100960007573653A206F6E0A000A6B6579626F6174
:1009700072643A206F66660A000A6B6579626F617D
:1009800072643A206F6E0A000A6D61747269783A77
:10099000206F66660A000A6D61747269783A206F8A
:1009A0006E0A000A64656275673A206F6E0A000A73
:1009B00064656275673A206F66660A000A0A626FAC
:1009C0006F746C6F616465722E2E2E2000433E2082
:1009D000006D6B5F776865656C5F74696D655F74EA
:1009E0006F5F6D6178203D2025640A006D6B5F7735
:1009F0006865656C5F6D61785F7370656564203DE7
:100A00002025640A006D6B5F74696D655F746F5FAC
:100A10006D6178203D2025640A006D6B5F6D617803
:100A20005F7370656564203D2025640A006D6B5F0F
:100A3000696E74657276616C203D2025640A006DD4
:100A40006B5F64656C6179203D2025640A006D6BE5
:100A50005F776865656C5F74696D655F746F5F6D06
:100A60006178203D2025640A006D6B5F77686565BD
:100A70006C5F6D61785F7370656564203D202564EF
:100A80000A006D6B5F74696D655F746F5F6D61788F
:100A9000203D2025640A006D6B5F6D61785F737087
:100AA000656564203D2025640A006D6B5F696E7486
:100AB000657276616C203D2025640A006D6B5F6471
:100AC000656C6179203D2025640A00776865726550
:100AD0002064656C74613A20637572736F723D2592
:100AE000642C20776865656C3D25640A5365652034
:100AF000687474703A2F2F656E2E77696B69706514
:100B00006469612E6F72672F77696B692F4D6F75FE
:100B100073655F6B6579730A000A092D204D6F7547
:100B200073656B6579202D0A4553432F713A09711E
:100B30007569740A313A0964656C6179282A313023
:100B40006D73290A323A09696E74657276616C2890
:100B50006D73290A333A096D61785F737065656456
:100B60000A343A0974696D655F746F5F6D61780A64
:100B7000353A09776865656C5F6D61785F7370659C
:100B800065640A363A09776865656C5F74696D65F6
:100B90005F746F5F6D61780A0A703A097072696EEE
:100BA000742076616C7565730A643A097365742004
:100BB00064656661756C74730A75703A092B310A45
:100BC000646F776E3A092D310A706775703A092B98
:100BD00031300A7067646F776E3A092D31300A0A36
:100BE0007370656564203D2064656C7461202A2003
:100BF0006D61785F7370656564202A202872657066
:100C0000656174202F2074696D655F746F5F6D611D
:100C100078290A004C25640A00214353315F45308E
:100C20005F25303258210A00152E11241FBECFEF48
:100C3000DAE0DEBFCDBF04B603FE41C080914004C0
:100C400090914104A0914204B09143048730904BAD
:100C5000A740B04BA1F510924004109241041092AD
:100C600042041092430414BE0FB6F894A8958091E4
:100C70006000886180936000109260000FBE109247
:100C800001081092000889E0E3E0F0E0809357004B
:100C9000E491E695E370E15080E090E1E33040F4C8
:100CA000F0E0EE0FFF1FEE5CFE4F8081918100C0EF
:100CB000E0E0F0E8E81BF90BF695E795099511E0FF
:100CC000A0E0B1E0E2E4F4E602C005900D92AA399A
:100CD000B107D9F724E0AAE9B1E001C01D92A03420
:100CE000B207E1F716E0C5E1D6E004C02197FE01A6
:100CF0000E940532C431D107C9F70E94602E0C94BE
:100D00001F327EC9823309F447C0F0F4843209F4FB
:100D10004BC070F48C3109F44DC020F48B3109F4D0
:100D20004DC008958D31F1F1833209F449C0089521
:100D30008B3209F447C018F48A3261F108958C327D
:100D400009F18D32C9F108958234D1F040F4843331
:100D500099F0A0F08A3311F18C33B1F008958B34FF
:100D6000B9F028F4833491F0843401F108958D347E
:100D7000F9F08136A9F0089580E1089588E1089599
:100D800080E2089588E2089580E3089588E3089555
:100D900080E4089588E4089580E5089587E508953E
:100DA0008AE608958FE5089587E1089585E6089518
:100DB0008EE608958FE6089581E508958FE1089500
:100DC00087E2089588E008958B35D9F058F4813191
:100DD00001F118F48E3089F00895833161F0843583
:100DE00071F00895823689F018F48E3560F0089518
:100DF0008C3769F0089581E1089584E508958BE5C5
:100E000008958DE508958AE608958EE0089587E7B0
:100E100008958FE00895863809F467C030F5873665
:100E200009F44DC088F48C3509F469C038F4883071
:100E300009F469C0873509F460C00895843609F45F
:100E400042C08536D1F10895873709F454C028F49B
:100E50008D36B9F18E3679F108958438B1F108F004
:100E600042C08C3709F44DC008958C38D1F168F434
:100E7000893889F128F4873851F1883851F108957B
:100E80008A3859F18B3859F108958F3881F028F458
:100E90008D3849F08E3849F00895813941F148F094
:100EA000823939F1089587E7089587E608958FE735
:100EB00008958BE7089585E608958DE6089582E606
:100EC000089584E608958EE608958CE7089582E0FB
:100ED00008958EE708958CE0089583E0089584E0F6
:100EE000089585E0089588E0089580E1089581E0FF
:100EF000089589E0089588E508958CE5089583E5CF
:100F0000089588E6089586E708958091D40380FFC8
:100F10000CC06091140170E07595679575956795A3
:100F20006115710549F1862F089581FF06C0609112
:100F3000140170E075956795F3CF6091140182FDFF
:100F40000BC09091D5039923A1F06091130180917A
:100F50001401961738F0682F70E06038710500F3BF
:100F60008FE70895899FC001112470E00E94F2313B
:100F7000F4CF61E070E0D7CF81E008958091D40391
:100F800080FF12C06091160185E0689FB0011124B6
:100F9000759567957595679560387105A8F5611524
:100FA0007105A1F1862F089581FF09C06091160196
:100FB00085E0689FB001112475956795EDCF82FF9C
:100FC00007C06091160185E0689FB0011124E4CF4D
:100FD0002091D5032223A9F090911501609116016B
:100FE00085E0689FB00111242917B0F6269FA00163
:100FF000279F500D1124692F70E0CA010E94F23121
:10100000CBCF65E070E0CECF8FE7089581E0089503
:101010009C014FB7F8948091DD039091DE03A0917D
:10102000DF03B091E0034FBF821B930B08952FB7EE
:10103000F8948091DD039091DE03A091DF03B091DD
:10104000E0032FBF0895829590E09C01220F331F8B
:10105000220F331F2C7C95958795959587958373E3
:10106000282B30E0C901880F991F8A7A359527957A
:101070002575822B08958F929F92AF92BF92CF9247
:10108000DF92EF92FF920F931F93CF93DF9300D0E5
:1010900000D01F92CDB7DEB76B837C838D838C81AC
:1010A0009D81892B39F05F3F19F481E04F3F19F0A2
:1010B00080E001C081E080FF14C080E090E00F90EC
:1010C0000F900F900F900F90DF91CF911F910F9184
:1010D000FF90EF90DF90CF90BF90AF909F908F9058
:1010E0000895852F90E0242F30E06B81662309F46A
:1010F00067C080904B0390904C03A0904D03B0903C
:101100004E03C090E403D090E503E090E603F09036
:10111000E703C828D928EA28FB286FE170E0A62F4A
:1011200046015701062E04C0B694A794979487945D
:101130000A94D2F780FE1DC0E52FE7708B01F3E023
:10114000000F111FFA95E1F70E0F111DB4E0000F0B
:10115000111FBA95E1F7E42FEF70E00FF12FF11DA9
:10116000EE0FFF1FE050F849059114910130110571
:1011700021F46150710998F6A0E0FC0174E0EE0FD3
:10118000FF1F7A95E1F7E15BFC4FE20FF31FA083AD
:1011900028E0A29FC00111245770850F911D24E003
:1011A000880F991F2A95E1F7E42FEF70E80FF92FC8
:1011B000F11DEE0FFF1FE050F849859194917FCF0C
:1011C000FC0164E0EE0FFF1F6A95E1F7E15BFC4F65
:1011D000E20FF31FA081DCCF41E050E060E070E05F
:1011E00004C0440F551F661F771F8A95D2F740959C
:1011F00050956095709580914B0390914C03A09110
:101200004D03B0914E0384239523A623B7238093E7
:101210004B0390934C03A0934D03B0934E0308955A
:1012200041E050E060E070E004C0440F551F661FCD
:10123000771F8A95D2F780914B0390914C03A09130
:101240004D03B0914E03842B952BA62BB72B809387
:101250004B0390934C03A0934D03B0934E0308951A
:1012600080914A0390911903981301C008958F5FEC
:101270008770FACF1F93CF93DF9300D000D01F92D7
:10128000CDB7DEB7942F4983252F5A836B837C8398
:101290008D834C815D8181E0452B31F02F3F19F426
:1012A00081E09F3F09F080E0182F117080FD2BC076
:1012B00049815A816B817C818D81DDDE292F2295C8
:1012C0002F702C3078F42A30A8F422502230C8F045
:1012D000812F0F900F900F900F900F90DF91CF9173
:1012E0001F9108952C3011F02F3091F793FB1127A7
:1012F00010F9EECF803C28F0803E50F3815F8330C0
:1013000038F311E0E5CF10E0E3CF1F93CF93DF93E5
:10131000E091CF03F091D003309779F0EC01188180
:1013200080910D039091D803892B812B88830480B1
:10133000F581E02DCE0109951883DF91CF911F91A2
:101340000895E091CF03F091D003309721F0019000
:10135000F081E02D099480E00895E8EDF0E08081CF
:101360008E7F80831092E2001092DA001092E100EA
:10137000A0EEB0E08C9181608C9380818F77808328
:1013800019BCA7EDB0E08C918E7F8C9380818F7E0D
:1013900080831092DE020895E0DFF89487E797E7F4
:1013A000909301088093000887E090EBDC01809324
:1013B000400490934104A0934204B093430488E115
:1013C0009CE00FB6F894A895809360000FBE9093B0
:1013D0006000FFCFFC0180910A0390910B038617F8
:1013E0009707A0F06115710529F49091E8009E77A8
:1013F0009093E80090E06115710551F4911108C0D7
:101400008091E80082FF35C080E00895BC01F2CFF2
:1014100080910C038823C9F18530C9F18091E800DF
:1014200083FD31C08091E80082FDEACF8091E80021
:1014300080FFE1CF2091F3008091F200322F282F1E
:101440006115710519F02830310558F091E0283008
:10145000310509F090E02091E8002E772093E80014
:10146000CACF81918093F100615071092F5F3F4F86
:10147000E7CF80910C03882341F0853041F08091C3
:10148000E80083FFBDCF81E0089582E0089583E006
:1014900008952091E4003091E50085E69091EC00FC
:1014A00090FF06C09091E80090FF06C080E008958C
:1014B0009091E80092FDFACF90910C03992391F05E
:1014C000953091F09091EB0095FD10C04091E400B3
:1014D0005091E5002417350709F381509A01F1F680
:1014E00084E0089582E0089583E0089581E00895FE
:1014F0008091040387FF13C08091E80082FF06C03B
:101500008091E8008B778093E80004C080910C0301
:101510008111F2CF089580910C038823D9F3809133
:10152000E80080FFF8CF8091E8008E77ECCF982F0D
:101530009093E900242F762F50E0891731F07091B5
:10154000EC002091ED005091F00021FD07C09F5F5D
:10155000973071F78093E90081E008953091EB00B6
:101560003E7F3093EB003091ED003D7F3093ED00F6
:101570003091EB0031603093EB007093EC002093DE
:10158000ED005093F0002091EE0027FDE0CF80E0C9
:1015900008950F931F93CF93DF93CDB7DEB7AA972C
:1015A0000FB6F894DEBF0FBECDBF80910C03882329
:1015B00009F447C11091E9001F708091EC0080FF91
:1015C00038C080E8182B1092E9008091E80083FF72
:1015D00035C1E4E0F3E08091F100819383E0EC30E9
:1015E000F807C9F780910503833009F46EC018F538
:1015F000813009F446C0823009F4D4C08091E800FB
:1016000083FF0EC180910403909105039A3008F086
:1016100007C1E92FF0E0E15FF44F0C940532E30BD2
:10162000090C100C090C100C6A0C8B0C100C890D99
:10163000960D80E0C7CF8A3009F4A4C08B3009F43E
:101640007AC08930D9F6809104038132B9F680914D
:10165000080390910903892B89F68091E800877F20
:101660008093E8008091E80082FF2AC08091F10019
:101670008093E0028091E8008B778093E80038DF68
:10168000BDCF80910403813A09F0B8CF8091E80082
:10169000877F8093E8008091080390910903892B4C
:1016A00059F060E090E080E070E094DE8091E80026
:1016B0008B778093E800A2CF60E281EE92E0F4CFD6
:1016C00080910C038111CECF99CF80910403813A90
:1016D00009F094CF8091080390910903892B99F424
:1016E0008091E800877F8093E8008091E80080FF88
:1016F000FCCF809112018093F1008091E8008E77F9
:101700008093E800F5DE809108039091090301972A
:1017100009F074CF8091E800877F8093E800809182
:10172000E80080FFFCCF809110018093F100809150
:10173000E8008E77A2CF80910403813209F05ECF5A
:101740008091080390910903892B51F48091E8005E
:10175000877F8093E800CCDE80910603809312019E
:101760008091080390910903019709F047CF809178
:10177000E800877F8093E800BBDE809106038093BA
:1017800010013CCF80910403813209F037CF809162
:10179000E800877F8093E800ABDE809107038093A9
:1017A000E1032CCF80910403813A09F027CF809187
:1017B000E800877F8093E8008091E80080FFFCCFFD
:1017C0008091E103B2CF803889F0823849F5809169
:1017D00008038F70873020F58093E9008091EB003B
:1017E00085FB882780F91092E90006C080910103EB
:1017F00090910203911182609091E800977F9093FD
:10180000E8008093F1001092F1008091E8008E775B
:1018100031C0282F2D7F21F48823F1F0823071F11F
:101820008091E80083FF0AC08091E800877F809361
:10183000E8008091EB0080628093EB001F701093B2
:10184000E900AA960FB6F894DEBF0FBECDBFDF91B8
:10185000CF911F910F91089580910603813001F778
:10186000933009F080E0809302031092E9008091A8
:10187000E800877F8093E8003BDED2CF80910603AB
:101880008111F3CF809108038F702FEF280F26303E
:1018900038F68093E9002091EB0020FFE6CF9330EB
:1018A00031F48091EB0080628093EB00DECF909169
:1018B000EB0090619093EB0021E030E001C0220F3B
:1018C0008A95EAF72093EA001092EA008091EB00F3
:1018D0008860EACF8111A4CF009106030F77809131
:1018E000E3008078802B8093E3008091E800877F7D
:1018F0008093E800FDDD8091E80080FFFCCF8091BF
:10190000E30080688093E30083E0011101C082E07E
:1019100080930C0385CF8058823008F081CF2091CE
:101920000603309107032C3DA3E03A0799F583E0C5
:101930008A838AE289834FB7F894DE01139620E008
:101940003EE0E32FF0E081E280935700E49120FF36
:1019500003C0E295EF703F5FEF708E2F90E0EA30AA
:10196000B8F0C7968D939D932F5F243151F74FBFE9
:101970008091E800877F8093E8006AE270E0CE0102
:10198000019628DD8091E8008B778093E80048CFAE
:10199000C096E8CF8091080390910903432F552703
:1019A0004330510509F44FC078F54130510509F431
:1019B00045C084E590E0E7E0F5E04230510509F0EC
:1019C0002FCF2091E800277F2093E80020910A0381
:1019D00030910B038217930708F49C0140E0211516
:1019E000310509F063C0411161C08091E80082FDBA
:1019F000C9CF80910C03882329F2853019F2809198
:101A0000E80083FFF2CFBECF4132510509F43FC059
:101A10004232510509F004CF8330910508F000CF20
:101A2000FC01EE0FFF1FE45EFE4F0190F081E02D00
:101A3000875E9E4FDC018C9190E01DC082E190E0BA
:101A4000EBE5F5E0BECF332721303105C1F060F082
:101A50002230310509F0E4CEEDE6F5E0E4918E2F79
:101A600090E0EDE6F5E007C0EDEAF5E0E4918E2FB9
:101A700090E0EDEAF5E0009709F4D2CEA2CFE3EAD8
:101A8000F5E0E4918E2F90E0E3EAF5E0F4CF8330C7
:101A9000910508F0C5CE880F991FFC01EE5DFE4F41
:101AA0000190F081E02D89E090E08BCF80910C03D4
:101AB000882309F467CF853009F464CF8091E8006A
:101AC00083FD60CF8091E80082FD8FCF8091E80098
:101AD00080FF85CF8091F3009091F20089279827AD
:101AE00089272115310519F08830910550F041E022
:101AF000089709F040E08091E8008E778093E80035
:101B00006ECF44914093F1003196215031090196F6
:101B1000E8CF803809F084CE8091E800877F8093F9
:101B2000E800809103038093F1006FCE811178CE9D
:101B300000910603023008F073CE8091E800877FA1
:101B40008093E80000930303D3DC002381F084E05A
:101B500080930C0342E261EC81E0E9DC42E061EC5D
:101B600082E0E5DC46E261EC83E0E1DC59CE809185
:101B7000E30087FDECCF81E0EBCFEF92FF920F9374
:101B80001F93CF937C018B0184DCC82F811117C078
:101B90008091E80085FD0BC08091E8008E778093EE
:101BA000E800F7DC76DC882399F3C82F08C0F7013A
:101BB00081917F018093F1000150110949F78C2F29
:101BC000CF911F910F91FF90EF900895CF92DF92E8
:101BD000EF92FF920F931F93CF93DF93C8EDD0E066
:101BE00088818F7E8883E7EDF0E08081816080834B
:101BF00084E082BF81E08093DE0288818E7F8883CB
:101C000002EE10E0F80110821092DA0081EEC82E88
:101C1000D12CF601108288818F7788838881806833
:101C2000888388818F7D888319BC10920C03109261
:101C30000303109202031092010390EEE92EF12C9F
:101C4000F70180818B7F808388818160888342E077
:101C500060E080E06CDCF60180818E7F8083F8019B
:101C6000808181608083808188608083F7018081AA
:101C70008E7F8083888180618883DF91CF911F91DF
:101C80000F91FF90EF90DF90CF9008958091E00248
:101C900008958091BA02811113C09FB7F8944091C2
:101CA000DD035091DE036091DF037091E0039FBF7D
:101CB000443C59406105710518F081E08093BA02F7
:101CC0000895FF920F931F93CF93DF93D82F0FB6F2
:101CD00007FE42C080910C03843079F080910301AB
:101CE00090E001962091050130E08223932320911A
:101CF00004012817190609F0CAC0CBDF81110FC0F3
:101D00008091030190E001962091050130E082234B
:101D10009323209104012817190609F0B8C087D928
:101D20008C01C091E900CF708091EC0080FD35C03E
:101D300080E0C82B83E08093E9008091EB0085FD73
:101D400008C08091EB0080FF04C08091EE0087FD09
:101D500045C0CF70C093E900E09103018E2F90E061
:101D600001962091050130E0822393232091040104
:101D70002817190609F484C080910101909102018D
:101D8000E80FF92FF11DD083809103018F5F9091AF
:101D9000050189238093030173C080E8CACFE091D5
:101DA0000101F0910201E80FF11D90818F5F2091F8
:101DB00005018223809304019093F1008091E80053
:101DC00085FD0CC08091E80080FF08C08091E8008C
:101DD0008E778093E80085E0809300018091040174
:101DE00090910301981739F19091E80095FDD7CFB4
:101DF00080E028C01092F10031C08091030190E092
:101E000001962091050130E0822393232091040163
:101E10002817190609F09DCFF0900001FF2009F462
:101E200098CF05D98017910709F487CFFA94F092DB
:101E300000018C0182CF8091E80085FFD9CFD0933B
:101E4000F10081E02091F3009091F200322F292FD0
:101E5000232B81F09091E80090FF0CC09091E80056
:101E600095FDC8CF9091E8009E779093E80095E0AB
:101E700090930001882309F4C0CFCF70C093E9008C
:101E800080E0DF91CF911F910F91FF900895E09135
:101E9000030172CF262F30E094E0359527959A956F
:101EA000E1F72770E62FEF70823079F08330B9F0D8
:101EB0008130F9F480E1289F90011124E20FF32F83
:101EC000F11DE15FFB4F8491089580E1289F90010F
:101ED0001124E20FF32FF11DE157FC4FF4CF80E105
:101EE000289F90011124E20FF32FF11DE15FFC4FB9
:101EF000EACF80E80895643808F0DCC0E62FF0E00F
:101F0000EC57F04F0C94053258105A105A104610E6
:101F100042105A105A105A105A105A105A1048109B
:101F200044105C105A105A1042100B105A105A10DC
:101F30005C1046105A105A1044105A105A105A1079
:101F40005A105A105A100810461058105A104010C3
:101F50005A105A105A101E1048105A105A10501089
:101F60005A105A105A1020104A105A103E105A1087
:101F700042105A105A1054104C105A104E1044105F
:101F80005A105A105A105210091015105A105A109F
:101F90005A105A105A105A1009105A1022105A107A
:101FA0005A1048105A105A104A105A105A105A1003
:101FB0005A105A105A105A105A105A1024105A1007
:101FC0005A105A1050105A105A105A105A105A10CB
:101FD0005A105A105A105A105A1026105A10281017
:101FE0002A105A105A105A102C102E1030105A1055
:101FF000321034105A1036105A10561038105A1029
:102000003C103A1036105A105A105A105A104A10F2
:1020100067E1862F0895FC018281938180599B4A54
:102020006FE00297B0F763E1F4CFFC018281938106
:1020300080599B4A029768F76CE7EBCF6FE1E9CFD5
:1020400067E2E7CF60E6E5CF62E6E3CF6CE5E1CF9C
:1020500063E5DFCF6FE2DDCF69E3DBCF67E3D9CFA5
:102060006FE3D7CF67E4D5CF6FE4D3CF60E0D1CFB4
:1020700066E5CFCF6EE5CDCF6FE7CBCF6EE6C9CFAC
:102080006FE6C7CF68E0C5CF60E1C3CF68E1C1CFDD
:1020900060E2BFCF68E2BDCF60E3BBCF68E3B9CFFA
:1020A00060E5B7CF67E5B5CF6FE5B3CF6DE6B1CFEC
:1020B00065E6AFCF6F77ADCF69E1ABCFFC0184812F
:1020C000E9DE87FD21C0E82FF0E094E0F595E79583
:1020D0009A95E1F7EE0FFF1FE554FD4F40815181C6
:1020E000282F2F7081E090E002C0880F991F2A9559
:1020F000E2F79C0124233523232B31F08095909522
:1021000084239523918380830895FC018481C2DE1A
:1021100087FD1FC0E82FF0E094E0F595E7959A95CC
:10212000E1F7EE0FFF1FE554FD4F40815181282F4D
:102130002F7081E090E002C0880F991F2A95E2F786
:102140009C0124233523232B21F4842B952B91836D
:1021500080830895EBEBF2E01182108213821282E9
:1021600015821482178216821186108613861286B3
:1021700015861486178616860895FC019CB3838DF8
:10218000982B9CBB9DB3838D892B8DBB0895FC013F
:102190008AB1948D909598239AB99BB1848D892B9F
:1021A0008BB90895FC018BB1938D909598239BB9C1
:1021B0008AB1938D892B8AB9CF01E9CFCF93DF9371
:1021C000EC012E9826982F982798ECDF898D843083
:1021D000F8F490916900880F22E030E001C0220FEE
:1021E0008A95EAF7892F822B809369009DB38B8DA6
:1021F000809589238DBB198218821A821B8280E008
:1022000090E89D838C831F821886DF91CF9108957B
:1022100090916A008370880F22E030E001C0220FA5
:102220008A95EAF7892F822B80936A00DFCFFC0121
:102230008BB1948D909598239BB99AB1848D892BFD
:102240008AB90895FC018AB1938D909598239AB923
:102250009BB1838D892B8BB90895CF93DF93EC01CC
:10226000F1DFCE01DF91CF9192CFCF93C82FE4EE73
:10227000E80FE83408F07FC0F0E0EF5BFE4E0C940E
:102280000532A111AF11BB11BB119311BB11BB11D1
:10229000BB11BB11BB11BB11BB11BB11BB11BB11DE
:1022A000BB11BB11BB119511BB119711BB11BB1118
:1022B000BB11BB11B311BB11C811B111BB11BB11C3
:1022C000BB11BB11BB11BB11BB11BB11BB11BB11AE
:1022D000BB11BB11BB118911A7119911AB11BB1116
:1022E0009B11BB119F11BB11A9119D11AD11A31120
:1022F000A511BB11BB11BB11BB11BB11BB11BB1194
:102300008D118F119111B511B711BB11BB11BB11FB
:10231000B911C5E58C2FCF910895CAE5FBCFCBE568
:10232000F9CFCCE5F7CFCDE5F5CFCEE5F3CFCFE5CF
:10233000F1CFC0E6EFCFC1E6EDCFC2E6EBCFC3E60B
:10234000E9CFCFE6E7CFC1E7E5CFC2E7E3CFC4E708
:10235000E1CFC5E7DFCFC7E7DDCFC8E7DBCFCAE70F
:10236000D9CFCCE7D7CFCFE7D5CFC0E7D3CFC9E719
:10237000D1CFCBE7CFCF1F92CF9389E19CE09F9342
:102380008F930E940C2E0F900F900F900F90C2CF42
:10239000C4E5C0CF8330C9F128F4813061F08230C8
:1023A00019F10895853009F452C008F43FC0863011
:1023B00009F45EC0089580911801681790F4861B97
:1023C00080931801809118011F928F938CEB9AE0F3
:1023D0009F938F930E940C2E0F900F900F900F9051
:1023E000089510921801EECF80911701681750F4EC
:1023F000861B80931701809117011F928F938AEAA1
:102400009AE0E6CF10921701F6CF80911601681777
:1024100050F4861B80931601809116011F928F93B2
:1024200087E99AE0D5CF10921601F6CF8091150179
:10243000681750F4861B80931501809115011F9237
:102440008F9382E89AE0C4CF10921501F6CF809165
:102450001401681750F4861B8093140180911401B5
:102460001F928F9389E69AE0B3CF10921401F6CFB2
:1024700080911301681750F4861B8093130180919B
:1024800013011F928F938EE49AE0A2CF1092130152
:10249000F6CF833009F445C028F4813061F08230F2
:1024A00049F10895853009F46AC008F451C08630B6
:1024B00009F47CC0089580911801482F460F5527D4
:1024C000551F4F3F510594F4680F60931801809198
:1024D00018011F928F938FE39AE09F938F930E942E
:1024E0000C2E0F900F900F900F9008958FEF809308
:1024F0001801EDCF80911701482F460F5527551F22
:102500004F3F510554F4680F6093170180911701F4
:102510001F928F938DE29AE0E0CF8FEF80931701A7
:10252000F5CF80911601482F460F5527551F4F3F75
:10253000510554F4680F60931601809116011F92A3
:102540008F938AE19AE0C9CF8FEF80931601F5CF80
:1025500080911501482F460F5527551F4F3F5105B4
:1025600054F4680F60931501809115011F928F93A9
:1025700085E09AE0B2CF8FEF80931501F5CF80917F
:102580001401482F460F5527551F4F3F510554F44E
:10259000680F60931401809114011F928F938CEE49
:1025A00099E09BCF8FEF80931401F5CF80911301B9
:1025B000482F460F5527551F4F3F510554F4680FBC
:1025C00060931301809113011F928F9381ED99E025
:1025D00084CF8FEF80931301F5CFCF93DF932091BA
:1025E0001003309111032817390701F1909311035B
:1025F00080931003E091CF03F091D0033097B1F0B6
:10260000EC010084F185E02D09958091E30385704C
:10261000853061F4DF93CF938FEB95E09F938F9399
:102620000E940C2E0F900F900F900F90DF91CF9182
:102630000895CF93DF9320910E0330910F03281755
:10264000390701F190930F0380930E03E091CF03BC
:10265000F091D0033097B1F0EC010680F781E02DC6
:1026600009958091E3038570853061F4DF93CF9302
:1026700081EB95E09F938F930E940C2E0F900F900B
:102680000F900F90DF91CF910895CF93DF93EC01DE
:102690008F8190E001968F70992728852817190659
:1026A00071F4198218821A821B8280E090E89D835F
:1026B0008C831F821886CE0160DDCE01CEDD2FB760
:1026C000F89488859F81981307C02FBFCFEFDFEF65
:1026D000CE01DF91CF910895FE01E80FF11D9185A4
:1026E0008F5F8F708887C92FD0E02FBF8091E30361
:1026F00080FFEECF1F929F938AE991E09F938F9383
:102700000E940C2E0F900F900F900F90E1CFEF9240
:10271000FF920F931F93CF93DF937C010E941708C2
:102720008C01F70180819181B0DFEC01019631F4D9
:10273000C8010E940808843F914098F3CE01DF91C0
:10274000CF911F910F91FF90EF90089589E19BE049
:102750000E94732D1F9281E08F931F9285E08F93CB
:102760008BEC9AE09F938F930E940C2E0F900F900A
:102770000F900F900F900F9008958091E30383FFC7
:102780007EC08BEC96E00E94732D8091D8031F923F
:102790008F9386EC96E09F938F930E940C2E84EC8F
:1027A00096E00E94732D8091D903282F082E000CEB
:1027B000330B3F938F9381EC96E09F938F930E940E
:1027C0000C2E8FEB96E00E94732D8091DA03282F58
:1027D000082E000C330B3F938F938CEB96E09F9366
:1027E0008F930E940C2E8AEB96E00E94732D8091AD
:1027F000DB03282F082E000C330B3F938F9387EBBE
:1028000096E09F938F930E940C2E85EB96E00E949A
:10281000732D8091DC03282F082E000C330B3F937F
:102820008F9382EB96E09F938F930E940C2E8FEAFA
:1028300096E00E94732D8091D5031F928F938CEAAE
:1028400096E09F938F930E940C2E8AEA96E00E9456
:10285000732D8091D4031F928F9387EA96E09F9304
:102860008F930E940C2E84EA96E00E94732D8DB700
:102870009EB74C960FB6F8949EBF0FBE8DBF88EDE5
:1028800093E00E9485090E9417089093D7038093D4
:10289000D6030895CF93DF938091D3039091D20311
:1028A000892B80939A029091D103992389F0892BE7
:1028B00080939A02EBE9F2E02AEB32E080E091911A
:1028C00091118F5F2E173F07D1F781111092D1031D
:1028D000E091CF03F091D0033097A1F10280F38112
:1028E000E02D8AE992E009958091E30382FF2AC0F6
:1028F00080FF04C089E996E00E94732DD0E0C0E01B
:102900008091E30380FF10C0FE01E656FD4F8081F9
:102910001F928F9383E996E09F938F930E940C2ED2
:102920000F900F900F900F902196C032D10541F774
:102930008091E30380FF06C081E996E0DF91CF91AB
:102940000C94732DDF91CF9108951092D3031092C0
:10295000D203EBE9F2E0119282E0EA3BF807D9F703
:1029600099DF85E0E8EDF3E0DF011D928A95E9F754
:102970001092D5031092D40300DF90E080E059DE7E
:1029800090E080E02ACECF93C82F1F928F9384E1EE
:102990009CE09F938F930E940C2E81E090E0A0E03A
:1029A000B0E004C0880F991FAA1FBB1FCA95D2F7B9
:1029B0008093E4039093E503A093E603B093E703C9
:1029C0000F900F900F900F90CF91BFCFC3DBBDDF63
:1029D00081EA91E09F938F930E940C2E0F900F90AD
:1029E0000895882339F080959091D30389238093AB
:1029F000D30350CF0895882331F09091D303892BCE
:102A00008093D30347CF0895882309F451C09CEFE6
:102A1000980F913A58F5909112019923D1F0909125
:102A200011019923B1F0E82FE695E695E695F0E0DF
:102A3000E656FD4F877021E030E0A90102C0440F47
:102A4000551F8A95E2F7CA01809591818923818378
:102A500021CFEAE9F2E028EB32E09281891301C04C
:102A6000128231962E173F07C1F7F2CF90E2980FEE
:102A7000983088F4877021E030E0A90102C0440F4B
:102A8000551F8A95E2F7CA0180959091D303892357
:102A90008093D303DDCF9BE5980F933018F490E03B
:102AA00080E0C7CD885A873118F490E080E095CD5A
:102AB0000895CF93873208F04FC08E3108F01DC1C2
:102AC000803109F4A6C0F8F4873009F485C048F4D1
:102AD000863009F46EC080EB97E00E94732DC0E051
:102AE00026C08B3009F460C08E30A9F79091E303C3
:102AF000892F8B7F92FF84608093E30382FF86C0DF
:102B000089E799E07AC0863109F4AAC098F4813146
:102B100011F71BDFC091110181E0C827C09311019B
:102B2000CC2309F4E7C08DEB97E00E94732D8C2F26
:102B3000CF910895893109F47CC08B3161F6909171
:102B4000E303892F8D7F91FF82608093E30381FFF0
:102B50005AC086E999E051C0883331F150F4893286
:102B600029F0853319F0873209F0B5CF80E00BDF0B
:102B700031C08334D9F328F48A3308F4ACCF8953B5
:102B8000F6CF883409F0A7CFE0DE8CEB99E00E9405
:102B9000732D2FEF83ED90E3215080409040E1F7BB
:102BA00000C000000E94CC098EEE96E00E94732DBA
:102BB00011C08091E303817F8E7F8093E30389E8D6
:102BC00097E00E94732D8DEC99E00E94732D81E0B7
:102BD0008093E203C1E0ABCF8091E30380FF0BC0A1
:102BE0008FEA99E00E94732D8091E303817F8E7FAD
:102BF0008093E303EFCF83EA99E00E94732D8091E5
:102C0000E3038160F5CF88E899E0D0CF89E699E0C9
:102C1000CDCF9091E303892F877F93FF88608093C6
:102C2000E30383FF03C08DE599E0E7CF80E599E0FA
:102C3000BDCF81E499E00E94732D8EE299E00E945D
:102C4000732D89EE98E00E94732D83EC98E00E942A
:102C5000732D8EE698E00E94732D83E498E0A6CF52
:102C600085E398E00E94732D0E94A1091F928F9323
:102C70008BE198E09F938F930E940C2E809112011C
:102C80001F928F9384E098E09F938F930E940C2E65
:102C90008091E1031F928F9381EF97E09F938F9331
:102CA0000E940C2E809111011F928F938EED97E060
:102CB0009F938F930E940C2E2FB7F8948091DD0381
:102CC0009091DE03A091DF03B091E0032FBFBF938B
:102CD000AF939F938F9387EC97E09F938F930E947E
:102CE0000C2E8DB79EB746960FB6F8949EBF0FBEBA
:102CF0008DBF70CF82EB97E059CF8D5138CFCF93F6
:102D0000882309F4ADC0C82F8CEF8C0F813A08F0EE
:102D10006BC18091E203813071F110F1823009F4CE
:102D200058C01092E20380911201882309F442C135
:102D300080911101882309F43DC1EC2FE695E695B9
:102D4000E695F0E0E656FD4FC77021E030E001C0A7
:102D5000220FCA95EAF78181822B8183CF919ACD88
:102D600080919A02823211F08434E9F68C2FA1DE30
:102D7000811176C0D8CF80919A028232B9F384341F
:102D8000A9F3C431C9F048F4CB3059F0C031C1F0D7
:102D90008FEC95E00E94732D11C0C93269F0C833E1
:102DA000B9F789E897E00E94732D85ED95E00E94C0
:102DB000732D81E08170DCCF1092E20380E0FACFC6
:102DC000C5DC81ED95E00E94732D82E08093E203E3
:102DD000F0CFC432C8F4CE3108F0BDC0CB30E1F042
:102DE00040F4C73009F4CCC08EE796E0CF910C9444
:102DF000732DC331B9F1C431B9F78091120388231F
:102E000041F11092120309C0CB3409F4B7C0B8F4F1
:102E1000C93299F3C83341F799DC809112038823B2
:102E200009F4C5C01F928F9388E796E09F938F9314
:102E30000E940C2E0F900F900F900F9011C0C13573
:102E400009F497C0C23509F48FC0CE3469F66AE040
:102E500091C08DE896E00E94732D81E08093E2039B
:102E6000CF91089587E696E00E94732D85E596E060
:102E70000E94732D809118011F928F9382E596E036
:102E80009F938F930E940C2E80E596E00E94732DF5
:102E90008EE396E00E94732D809117011F928F930D
:102EA0008BE396E09F938F930E940C2E89E396E02C
:102EB0000E94732D8AE296E00E94732D8091160184
:102EC0001F928F9387E296E09F938F930E940C2E20
:102ED00085E296E00E94732D84E196E00E94732DB6
:102EE000809115011F928F9381E196E09F938F93BC
:102EF0000E940C2E8FE096E00E94732D8AEF95E0E1
:102F00000E94732D809114011F928F9387EF95E09B
:102F10009F938F930E940C2E85EF95E00E94732D56
:102F20008EED95E00E94732D809113011F928F9377
:102F30008BED95E09F938F930E940C2E89ED95E089
:102F40000E94732D8DB79EB748960FB6F8949EBF1A
:102F50000FBE8DBF62CFCE51EC2FF0E0E85DFE4F8B
:102F600080818093120359CF61E08091120391DA3E
:102F700054CF61E0809112030DDA4FCF6AE0F5CFB4
:102F80008EE18093180182E3809317018AE0809399
:102F9000160184E18093150188E08093140188E292
:102FA0008093130180E896E00E94732D36CF85E769
:102FB00096E01CCFACE9B2E0EFEF80E09D91C9173D
:102FC00009F4CCCEEF3F19F4911101C0E82F8F5FC7
:102FD0008E31A1F7EF3F09F4C1CE0E2E000CFF0B8E
:102FE000E656FD4FC283BACE80E28C0F883068F47B
:102FF000C77021E030E001C0220FCA95EAF7809146
:10300000D303822B8093D303A9CE8BE58C0F83301F
:1030100060F481E890E0C53A31F083E890E0C63A88
:1030200011F482E890E0CF9104CB88E58C0F8731D2
:1030300008F067C082EE90E0C83A09F460C089EEFB
:1030400090E0C93A09F45BC08AEE90E0CA3A09F40C
:1030500056C085EB90E0CB3A09F451C086EB90E086
:10306000CC3A09F44CC083EB90E0CD3A09F447C068
:1030700084EB90E0CE3A09F442C087EB90E0CF3A7F
:10308000F1F18CEC90E0C13BD1F18DEC90E0C03BD4
:10309000B1F183E891E0C23B91F18AE891E0C33B52
:1030A00071F182E991E0C43B51F184E991E0C53BC3
:1030B00031F181E292E0C63B11F183E292E0C73B3D
:1030C000F1F084E292E0C83BD1F085E292E0C93BA6
:1030D000B1F086E292E0CA3B91F087E292E0CB3B0E
:1030E00071F08AE292E0CC3B51F08FE690E0CD3B6C
:1030F00031F090E080E0CE3B11F480E790E0CF919A
:103100006CCACF3B09F0ACCE20DC9FEF20E782E019
:10311000915020408040E1F700C000000E94CC099F
:10312000CF92DF92EF92FF920F931F93CF93DF9393
:1031300000D000D01F92CDB7DEB76C0185E0F6015C
:10314000DE01119601900D928A95E1F7F60140811A
:1031500051812381348191E02115310531F05F3FA8
:1031600019F491E04F3F09F090E090FD94C0F60112
:103170000281F580F2949FE0F92249835A830B8300
:10318000722F3D832C83602F8D810E943B08182F66
:10319000E92FE295EF70EF3008F07DC0F0E0ED52DE
:1031A000F74E0C940532E218E2181C191C198F19FD
:1031B000BF194B194B19B01A4B19861B861B4B199B
:1031C0004B19411CF92FFF70FF2E907F19F0F294DC
:1031D00080EFF8220023B9F0FF2031F08091D20374
:1031E000F82AF092D20356DB812F0F900F900F90A8
:1031F0000F900F90DF91CF911F910F91FF90EF9063
:10320000DF90CF907CCD812FFFDBFF2009F443C0FE
:10321000F0948091D203F822F092D2030F900F9095
:103220000F900F900F90DF91CF911F910F91FF9012
:10323000EF90DF90CF902ECB892F8F70907F9032C0
:1032400011F08295807F112379F0113009F447C085
:10325000002309F453C0FF2059F0F601958190FF37
:1032600063C29F70958304C0002319F1F1100EC052
:103270000F900F900F900F900F90DF91CF911F91B3
:103280000F91FF90EF90DF90CF90B5CB21E0F2123D
:10329000EFCF8093D1030F900F900F900F900F906E
:1032A000DF91CF911F910F91FF90EF90DF90CF9022
:1032B0000895F11010C01092D1030F900F900F904D
:1032C0000F900F90DF91CF911F910F91FF90EF9092
:1032D000DF90CF9086CB91E0F912EDCFDCCF0023C9
:1032E00049F0E5E0EF15B8F29091D303982309F483
:1032F000BFCFE3CFF4E0FF1570F2DFCFFF20E9F29C
:10330000812F0F900F900F900F900F90DF91CF9122
:103310001F910F91FF90EF90DF90CF9075CB892F89
:10332000869586958370B9F0813009F0B4CF812FEE
:103330009370011102C090E080E00F900F900F9009
:103340000F900F90DF91CF911F910F91FF90EF9011
:10335000DF90CF9042C9812F9370011102C090E09D
:1033600080E00F900F900F900F900F90DF91CF9112
:103370001F910F91FF90EF90DF90CF905AC90023DB
:1033800009F470C0803F99F40E94BE078195809334
:10339000DA030F900F900F900F900F90DF91CF9165
:1033A0001F910F91FF90EF90DF90CF90E6C9813F82
:1033B00019F40E94BE07EBCF823F31F40E94BE0792
:1033C00081958093D903E5CF833F19F40E94BE070E
:1033D000F8CF893F29F40E9485078093DB03D9CF7A
:1033E0008A3F21F40E9485078195F7CF8B3F31F406
:1033F0000E94850781958093DC03CBCF8C3F19F425
:103400000E948507F8CF8091D8038160143FA1F016
:103410008091D8038260153F79F08091D803846051
:10342000163F51F08091D8038860173F29F0183F6C
:1034300031F48091D80380618093D803AACF809122
:10344000D40381601D3F59F08091D40382601E3FF8
:1034500031F01F3F09F09DCF8091D40384608093A9
:10346000D40397CF803FC1F48091DA0387FD109297
:10347000DA038091D90381118CCF8091DA03811115
:1034800088CF8091DB03811184CF8091DC0381118F
:1034900080CF1092D5037DCF813F29F48091DA034C
:1034A00018162CF3E6CF8091D903123F29F487FF39
:1034B000E0CF1092D903DDCF133F19F41816CCF3E7
:1034C000D8CF193F39F48091DB03181694F6109287
:1034D000DB03CFCF1A3F29F48091DB0387FFC9CFED
:1034E000F6CF1B3F39F48091DC0387FFC2CF1092E7
:1034F000DC03BFCF1C3F29F48091DC031816BCF31A
:10350000B8CF8091D8038E7F143FA1F08091D8036B
:103510008D7F153F79F08091D8038B7F163F51F056
:103520008091D803877F173F29F0183F31F48091AD
:10353000D8038F7E8093D8039CCF8091D4038E7F55
:103540001D3F59F08091D4038D7F1E3F31F01F3F06
:1035500009F08FCF8091D4038B7F8093D40389CFE0
:10356000892F837009F064C0011195CE812F829557
:1035700086958770880F880F412F4F70C42ED12CED
:10358000F12CE12C082E04C0CC0CDD1CEE1CFF1C21
:103590000A94D2F740E050E0BA0114FF11C00FE0E6
:1035A00010E020E030E004C0000F111F221F331F85
:1035B0008A95D2F7B901A80140955095609570950C
:1035C0000091E4031091E5032091E6033091E703B5
:1035D0009695969593709230E9F028F5913089F0A0
:1035E0004C295D296E297F294023512362237323AF
:1035F0004093E4035093E5036093E6037093E7037D
:103600004ACEC02AD12AE22AF32A4C295D296E2902
:103610007F29EECF4C295D296E297F29402751272C
:1036200062277327E5CF4023512362237323EDCF15
:103630008695002311F0892F8170882309F42BCE01
:10364000812F829586958770880F880F412F4F7044
:10365000C42ED12CF12CE12C082E04C0CC0CDD1C86
:10366000EE1CFF1C0A94D2F740E050E0BA0114FFB0
:1036700011C00FE010E020E030E004C0000F111F87
:10368000221F331F8A95D2F7B901A80140955095A2
:103690006095709500914B0310914C0320914D0360
:1036A00030914E039695969593709230E9F028F5F7
:1036B000913089F04C295D296E297F2940235123BF
:1036C0006223732340934B0350934C0360934D0349
:1036D00070934E03E0CD0C291D292E293F29402B44
:1036E000512B622B732BEECF4C295D296E297F293C
:1036F0004027512762277327E5CF402351236223B8
:1037000073234C295D296E297F29DCCF803F09F482
:103710004DC0C8F480E4810F803268F1002309F4C1
:10372000ABC0FF2009F4A5C0812FE9DA193309F0F5
:1037300099C0FFEF21EE84E0F15020408040E1F796
:1037400000C00000A8CD823F09F470C008F45BC03F
:10375000833F21F7002309F47CC0292F2F7181E0DA
:1037600090E0A0E0B0E004C0880F991FAA1FBB1F23
:103770002A95D2F73AC0E12FE071FE2E892F8F7182
:10378000002351F00E941009812F8295807FF11053
:103790006FCD812F8F706CCD0E94EC08812F8295A8
:1037A000807FF1108ACD812F8F7087CD002331F17A
:1037B000F4E0FF1508F46FCD292F2F7181E090E020
:1037C000A0E0B0E004C0880F991FAA1FBB1F2A9574
:1037D000D2F740914B0350914C0360914D0370918F
:1037E0004E0384279527A627B72780934B039093F2
:1037F0004C03A0934D03B0934E034DCD25E02F1500
:1038000008F449CDD9CF892F8F71002399F00F90FB
:103810000F900F900F900F90DF91CF911F910F910C
:10382000FF90EF90DF90CF900C941009892F8F714B
:10383000002369F30F900F900F900F900F90DF917E
:10384000CF911F910F91FF90EF90DF90CF900C944C
:10385000EC0810924B0310924C0310924D031092FF
:103860004E0319CD133509F464CF173409F013CD85
:1038700060CF892F8F71CBCFF11042CD892F8F71FF
:10388000D9CF811108CD002309F405CD5ED88FEF83
:1038900090E7E2E081509040E040E1F700C0000096
:1038A0000E94CC09CF93DF9380911803807FB1F4FD
:1038B00080911503882391F080914A03D0911903D8
:1038C00040911303509114036091160370911703F4
:1038D000C1E04F3F09F0C0E0D81303C0DF91CF91A2
:1038E000089521E06115710521F02C2F5F3F09F04B
:1038F00020E090E020FD31C026E0289FF001299FC4
:10390000F00D1124DF01A65EBC4F11962C9111978A
:10391000251323C02C91241320C012962C911297AA
:1039200021111BC013962D913C91261B370B283C6F
:10393000310598F4809118038F708061809318038B
:10394000E15EFC4F80818F708061808383E193E032
:10395000E7DBDF91CF910C94300901968770BCCFE3
:103960009F92AF92BF92CF92DF92EF92FF920F930E
:103970001F93CF93DF93CDB7DEB761970FB6F8945F
:10398000DEBF0FBECDBF8C0185E0F801DE011D96C4
:1039900001900D928A95E1F7F80140815181F28002
:1039A000C380D48090911303609114032091160377
:1039B0003091170381E02115310531F06F3F19F483
:1039C00081E09F3F09F080E0F82FF1709F2E80FD8D
:1039D0003FC183E1A82E83E0B82EE0901503F601E5
:1039E000E21BF30BEE2009F4F8C080911803782F46
:1039F000707FE83CF10508F0B4C071117DC0EF2C78
:103A0000651321C094131FC0F1101DC08F70806119
:103A100080931803C50184DB80911803F801858326
:103A20008E2D61960FB6F894DEBF0FBECDBFDF912D
:103A3000CF911F910F91FF90EF90DF90CF90BF90AB
:103A4000AF909F90089581E0C114D10431F05F3FA1
:103A500019F481E04F3F09F080E080FD14C081E05F
:103A60008F25F82FF170BF2EE0914A0320911903A2
:103A700080FD1FC0FF20A1F2809118038160809318
:103A80001803E12CCDCF80E0ECCF8E2F90E036E014
:103A9000E39FF0011124E65EFC4F3181531306C011
:103AA0003081431303C032813F11E4CFFC013196D2
:103AB000E770E213EACF7C2DD98AC88A6F2D8989F5
:103AC0000E943B08292F22952F70223050F024307D
:103AD00078F49F7051F0F8019581907F31F4E92CD2
:103AE0009FCF9F7011F08823D1F3805E8830B8F3A8
:103AF000C80116DB9B2CF3CF651306C0941304C0DA
:103B0000F801FF2009F484C04D875E87FF867C2D75
:103B1000D98AC88A6F2D89890E943A09882309F4B5
:103B2000A5C0FF2009F4A2C080911803803268F07C
:103B3000209113033091140338872F831986DB8675
:103B4000CA868C87CE010796EBDA86E0F801A3E1FE
:103B5000B3E001900D928A95E1F7A4DEEE24E394A0
:103B60005FCF711109C083E193E0DADA86E0F501F5
:103B700011928A95E9F785CF65130EC094130CC096
:103B8000F1100AC0F8018583C801CADA86E0F501A0
:103B900011928A95E9F744CF4D875E87FF867C2D89
:103BA000D98AC88A6F2D89890E943A09882309F425
:103BB0005DC0FF2009F45AC080911803803228F2BA
:103BC00020911303309114033A8329831B82DD82F1
:103BD000CC828E83CE010196B7CFE83CF105B0F6DA
:103BE000EF2CFF2009F442C065131EC094131CC0C3
:103BF0008091180380FD0FC0982F907F61F0F8012D
:103C00008583903F31F0982F907F905F8F70892B44
:103C10008583C80185DA86E0F801A3E1B3E001906D
:103C20000D928A95E1F7FCCE4D875E87FF867C2D4D
:103C3000D98AC88A6F2D89890E943A09811185CF56
:103C400080911803816080931803C80169DAE8CE77
:103C5000FF2061F04D875E87FF867C2DD98AC88A58
:103C60006F2D89890E943A0981116FCFC80158DAF6
:103C700075CFCF93DF93CDB7DEB767970FB6F894C4
:103C8000DEBF0FBECDBF4B8B5C8B6D8B7E8B8F8B66
:103C90001A8A198A85E0FE017396DE011D9601904D
:103CA0000D928A95E1F786E0FE013D96DE011796BA
:103CB00001900D928A95E1F7CE01079651DE8111B0
:103CC00037C086E0FE013796DE01119601900D9215
:103CD0008A95E1F79F8188852A853B85232B39F0DA
:103CE0008F3F19F481E09F3F19F080E001C081E02F
:103CF00080FD1EC02091190330E0C9010196877034
:103D0000992740914A034817190651F196E0929F6E
:103D1000D001939FB00D1124A65EBC4FFE013196D9
:103D200001900D929A95E1F7809319030E94300952
:103D300080914A03909119038917F9F0B6E08B9F9F
:103D4000C0011124865E9C4F0BDE8823B1F0809168
:103D50004A0390E001968770992780934A03E8CF41
:103D60000E94A5141092190310924A0386E0E3E121
:103D7000F3E0DF011D928A95E9F767960FB6F89494
:103D8000DEBF0FBECDBFDF91CF910895CF93DF93FC
:103D900000D01F92CDB7DEB720910C03243041F53F
:103DA00020911001222321F123E029839B838A8320
:103DB00082E08093E9008FEF9091E800815095FDBB
:103DC00006C095ED9A95F1F700008111F5CF80912D
:103DD000E80085FF0DC050E040E063E070E0CE01F8
:103DE00001960E94BD0D8091E8008E778093E800D7
:103DF0000F900F900F90DF91CF910895CF93DF93A5
:103E000000D01F92CDB7DEB720910C03243081F58E
:103E100020911001222361F119821A821B8222E073
:103E200029838138910520F0805891099B838A83EA
:103E300082E08093E9008FEF9091E800815095FD3A
:103E400006C095ED9A95F1F700008111F5CF8091AC
:103E5000E80085FF0DC050E040E063E070E0CE0177
:103E600001960E94BD0D8091E8008E778093E80056
:103E70000F900F900F90DF91CF91089520910C0338
:103E8000243049F522E02093E9002FEF3091E8003B
:103E9000215035FD06C035ED3A95F1F700002111AE
:103EA000F5CF2091E80025FF16C02091100150E0C9
:103EB00040E063E070E0222339F021E02093F1003C
:103EC00050E040E065E070E00E94BD0D8091E800A8
:103ED0008E778093E8000895CF93DF9320910C03B1
:103EE0002430D9F4EC01809112018823F1F0809103
:103EF00011018823D1F081E08093E90081E88150AD
:103F000021F09091E80095FF0BC08091E80050E00F
:103F100040E060E270E085FD1AC0DF91CF91089526
:103F20009AE29A95F1F700C0EACF81E08093E90028
:103F300081E8815021F09091E80095FF19C08091AF
:103F4000E80085FFEACF50E040E068E070E0CE0195
:103F50000E94BD0D8091E8008E778093E80080E29A
:103F6000FE01A1EEB2E001900D928A95E1F7D5CF66
:103F7000EFE3F1E03197F1F700C00000DACFCF9323
:103F8000DF93EC0199B14A8D8091DD032C813D8155
:103F90002115304849F58E832C813D813695279532
:103FA0003D832C8321E030E001C0220F4A95EAF7DF
:103FB000892F822329F08C819D8190689D838C8339
:103FC0008C819D81992780359105D1F170F58031E3
:103FD0009105B1F108F5892B29F11A828C819D8117
:103FE0009983888380E809C02E81821B8530A0F2E6
:103FF0008C819D819983888380E28B839BB18B8D9B
:10400000809589238BB98AB19B8D892B8AB980E0F1
:1040100090E89D838C8306C08032910519F080342E
:104020009105D9F6DF91CF910895803A910509F471
:1040300062C090F480389105A9F38039910569F642
:104040008C819D81998388838C819D8180399A4A56
:1040500009F080C082E0D1CF803C910521F0803D05
:10406000910571F3BACF8C819D81998388838C816E
:104070009D81892F99279D838C8382E28A838A81FF
:1040800084FF12C09BB18B8D809589238BB98AB137
:104090009B8D892B8AB987E592E00197F1F700C0E3
:1040A0000000CE010E9422112C813D818F81FE01F2
:1040B000E80FF11D21878F5F8F708F8390E001964D
:1040C0008F70992728852817190671F49DB38B8D59
:1040D000809589238DBB9BB18B8D809589238BB96E
:1040E0008AB19B8D892B8AB99F81888598138FCF40
:1040F00080E48B838CCF8A81811124C084E699B1BE
:104100002B8D922369F4882359F095E09A95F1F765
:1041100000008150F4CF25E02A95F1F7000081508E
:1041200099B12B8D922399F08111F5CF8C819D81CE
:10413000998388838C819D81892F99279D838C8386
:1041400081E29CCF8A81813209F06CCFEFCF81115F
:1041500069CFECCF8C819D812C813D8196FB882796
:1041600080F956E0369527955A95E1F78227282F52
:1041700030E0982F9E7F21F0359527958170F6CFFE
:10418000811102C081E039CF8C819D8197FF0CC0E5
:1041900080E18A838C819D8126E0969587952A957A
:1041A000E1F79D838C836BCF81E1F3CF0F931F9356
:1041B000CF938C01CAE1C15069F0C8010E94451338
:1041C0008F3F980749F48FE99FE00197F1F700C00E
:1041D0000000F1CF8FEF9FEFCF911F910F910895C6
:1041E000FC018AB1948D909598239AB98BB1948DE6
:1041F000892B8BB985E08A95F1F7000099B1848D00
:10420000982381E009F480E00895FC018AB1938D40
:10421000909598239AB98BB1938D892B8BB985E0B2
:104220008A95F1F7000099B1838D982381E009F414
:1042300080E008950F931F93CF93DF938C01EB01E0
:10424000C801E3DF811108C0209731F085E08A952D
:10425000F1F700002197F4CFCE01DF91CF911F91AC
:104260000F9108950F931F93CF93DF938C01EB0170
:10427000C801CBDF882341F0209731F085E08A9593
:10428000F1F700002197F4CFCE01DF91CF911F917C
:104290000F910895DF92EF92FF920F931F93CF93A8
:1042A000DF93EC01D62E1B828091E30380FF0CC0CC
:1042B0001F926F9383E991E09F938F930E940C2E3E
:1042C0000F900F900F900F908C819D8181159048D9
:1042D000E1F08091E30380FF0EC08C819D819F936C
:1042E0008F9389E891E09F938F930E940C2E0F90FB
:1042F0000F900F900F908FEF9FEFDF91CF911F9155
:104300000F91FF90EF90DF9008959DB38B8D809576
:1043100089238DBB8BE0E82EFF24F394CE010E940D
:10432000D2108FE193E00197F1F700C00000CE01B9
:104330000E9417118FE193E00197F1F700C0000090
:10434000CE010E94221168E97AE3CE018BDF892B2E
:10435000C1F481E08B838B81813009F0BEC0EA9487
:10436000EE2009F4BAC01B828091E30380FFD6CF10
:1043700086E891E09F938F930E940C2E0F900F90F0
:10438000CDCF10E000E090E59A95F1F78D2D90E00B
:10439000002E02C0959587950A94E2F780FF0DC024
:1043A00081E0F826CE010E94C71062E370E0CE01E2
:1043B00041DF892B31F482E0CDCFCE010E9417116D
:1043C000F4CF62E370E0CE014DDF892B11F483E07E
:1043D000C1CF0F5F1F4F08301105A9F620E52A95C0
:1043E000F1F7CE01FF2051F00E94C71062E370E0A8
:1043F000CE0120DF892B29F484E0ACCF0E94171175
:10440000F5CF62E370E0CE012DDF892B11F485E05A
:10441000A1CF80E58A95F1F7CE010E94C7100CE28A
:1044200011E0CE01DDDE882351F00115110549F0C0
:1044300095E09A95F1F7000001501109F2CF012B98
:1044400011F486E087CF0CE211E0CE01C9DE8111C4
:104450000AC00115110549F025E02A95F1F7000081
:1044600001501109F2CF012B11F487E073CF6CE2F8
:1044700071E0CE01DFDE892B11F488E06BCF8A81F9
:1044800084FF12C080E58A95F1F79BB18B8D8095F2
:1044900089238BB98AB19B8D892B8AB987E592E0F4
:1044A0000197F1F700C00000198218821A821B825E
:1044B00080E090E89D838C831F821886CE010E9445
:1044C0002D11CE010E94BD10CE01DF91CF911F9121
:1044D0000F91FF90EF90DF9069CE8C819D81998341
:1044E00088838B8180618B83CE010E94D2108FE301
:1044F0009FE10197F1F700C00000CE010E942D114D
:10450000CE010E94BD10F7CE0F931F93CF93DF9380
:104510008C01EB0169EEFC0180819181BBDEF80129
:104520008081918143DE8883F801808191813EDE24
:104530008983F8018081918139DE8A8399279F934D
:104540008F9389811F928F9388811F928F938FE819
:1045500094E09F938F930E940C2E8DB79EB7089680
:104560000FB6F8949EBF0FBE8DBFDF91CF911F9104
:104570000F9108950F931F93CF93DF93FC01A081B8
:10458000B18112968C911297813139F112968C91EA
:104590001297813229F112968C911297823219F179
:1045A0008F0162EFCD0176DE8F3F9807F9F08A3FE9
:1045B0009105F9F4C8010E9487138F3F9807E1F035
:1045C000D82FCC27C8010E9487139E01282BC90130
:1045D000DF91CF911F910F9108958DEF9FEFF8CF4D
:1045E0008CEF9FEFF5CF8BEF9FEFF2CF8FEF9FEF29
:1045F000EFCF8EEF9FEFECCF90E080E0E9CF0F930D
:104600001F93CF93FC0124812230C0F02430B1F0FD
:1046100062FBCC27C0F960FDC26061FDC460FC0193
:10462000008111816DEEC80135DE8A3F910531F4BC
:104630006C2FC801CF911F910F912CCECF911F915C
:104640000F910895CF93C82F682F86EF93E0D7DF9F
:104650006C2F88EE93E0CF91D2CFAF92BF92CF92E2
:10466000DF92EF92FF920F931F93CF93DF9300D0CF
:1046700000D01F92CDB7DEB78C01DC01ED91FC912B
:104680008381882369F1E080F180D3800E9417083C
:10469000FF92EF921F92DF929F938F9388EF92E0A9
:1046A0009F938F930E940C2ED801ED91FC9111974E
:1046B000838180750FB6F894DEBF0FBECDBF51F475
:1046C0008CE018968C9318978381823019F48DE0D2
:1046D00018968C931382D801ED91FC91118210826F
:1046E000D801ED91FC9111978281882309F443C090
:1046F000928115968C919817F1F1E080F180D2802B
:104700000E941708FF92EF921F92DF929F938F9360
:1047100081EE92E09F938F930E940C2EF801858189
:104720000FB6F894DEBF0FBECDBF0190F081E02D33
:1047300085FF03C0928194FD05C084FF13C0828170
:1047400085FF10C0D80118968C918B3059F48AEDF2
:1047500092E09F938F930E940C2E8CE0F80180874B
:104760000F900F90D801ED91FC91119782811596D1
:104770008C9311821082D8011896EC911897EE3024
:1047800008F04EC0F0E0E953FC4D0C940532D523FF
:10479000FD2321243C2452245D248C24A424C824F9
:1047A000E72420264D26BA2BA22B0E9417089F93A0
:1047B0008F9385ED92E09F938F930E940C2E0E9421
:1047C0001708F801978386830190F081E02D11820C
:1047D00010821282138280E090E89583848317828E
:1047E0001086D801ED90FC90C7010E94BD10C70152
:1047F0000E942D1181E0F80189C0D8018D919C9112
:104800000E9445130196C9F7F801868197810E949D
:104810000808893B9B4020F082E0D80118968C93D1
:1048200081E00F900F900F900F900F90DF91CF913C
:104830001F910F91FF90EF90DF90CF90BF90AF90BE
:1048400008950E9417089F938F9380ED92E09F93A5
:104850008F930E940C2E6FEFF801808191811ADDF9
:104860000F900F900F900F908A3F910511F486E002
:10487000D4CF83E0F80114C0ED91FC918DB3938DFA
:10488000909598239DBBCF010E94D2102E98269A16
:104890002F98279A0E941708F8019783868384E04F
:1048A0008087BECF16968D919C910E940808853F07
:1048B000914008F4B5CF85E0DDCF2E9826982F984B
:1048C0002798ED91FC911197118210821282138228
:1048D00080E090E89583848317821086ED90FC90A9
:1048E000C7010E94BD10C7010E942D110E94170828
:1048F0009F938F938BEC92E09F938F930E940C2E4B
:104900000E941708F8019783868386E080870F90BE
:104910000F900F900F9084CF8D919C910E94451322
:10492000019609F47DCF0E9417089F938F9386EC20
:1049300092E09F938F930E940C2E0E941708F8011B
:104940009783868387E0E2CF16968D919C910E9493
:104950000808853F914018F089E0F8018087D80168
:104960008D919C910E944513019609F459CF0E94A4
:1049700017089F938F9381EC92E09F938F930E94EF
:104980000C2E0E941708F8019783868388E0BECF1B
:1049900016968D919C910E940808853F914018F0D1
:1049A00089E0F8018087D8018D919C910E94451380
:1049B000019609F435CF0E9417089F938F938CEBD3
:1049C00092E09F938F930E940C2E89E014CFC80130
:1049D000D1DDD80113969C938E9312970E941708ED
:1049E0009F938F9387EB92E09F938F930E940C2E5F
:1049F000F801828193810F900F900F900F90009794
:104A000069F582E0D80114968C93F8018281938134
:104A100028E331E08F3F980709F4E1C08E3F2FEF84
:104A2000920709F4DAC08D3F3FEF930709F4F9C00C
:104A30002BE431E08C3FAFEF9A0709F4D0C020E5BA
:104A400031E08B3FBFEF9B0709F4C9C027E531E098
:104A5000009709F4C4C02AE431E0C1C08F3F980731
:104A600021F481E0F8018483D0CF9C012D5F3F4F7A
:104A70002230310530F22E5F3F4F2230310588F36E
:104A80008F3F910511F484E0BDCF9C0125583B4A2E
:104A90002230310520F08239BBEA9B07A1F460EF98
:104AA000F80180819181F6DB8A3F910509F0A9CF59
:104AB00063E0D8018D919C91EDDB8A3F910509F06F
:104AC000A0CF83E0CFCF9C0120593B4A2230310553
:104AD00008F051C089EA92E09F938F930E940C2EB8
:104AE00082E0D80114968C93149760EF8D919C917D
:104AF000D1DB0F900F908A3F9105D1F089E992E0C8
:104B00009F938F930E940C2E0F900F90F80182813B
:104B1000938181399B4A09F078CF60EFF801808159
:104B20009181B8DB8A3F9105A1F081E992E00AC04A
:104B300062E8D8018D919C91ADDB8A3F9105F1F639
:104B400085E992E09F938F930E940C2E0F900F9017
:104B50005CCF63E0D8018D919C919CDB8A3F9105ED
:104B600021F78DE892E09F938F930E940C2E83E0B3
:104B7000F8018483EBCF803BFFEB9F0709F4A1CFC3
:104B8000882781152BEA920709F43BCF81153FEB6B
:104B9000930709F496CF81159F4709F492CF81E7D7
:104BA00092E09F938F930E940C2E60EFF80180811A
:104BB000918170DB0F900F908A3F910529F060EF93
:104BC000D8018D919C916FCF62E0F8018081918135
:104BD00061DB8A3F910599F714CF2EE331E0F801AC
:104BE0004481413009F1423011F1433019F1443030
:104BF00021F54DE651E03F932F935F934F939F93A1
:104C00008F9381E692E09F938F930E940C2E8AE00F
:104C1000D80118968C930FB6F894DEBF0FBECDBFA7
:104C2000FFCD25E431E0DBCF4EE551E0E4CF41E6B6
:104C300051E0E1CF44E651E0DECF49E351E0DBCF84
:104C40000E9417089F938F938CE592E09F938F9318
:104C5000E3D70F900F900F900F90D80114968C917E
:104C60001497833009F440C0843009F443C0823083
:104C700019F40E94A109E6DC8BE0D80118968C9308
:104C80000E9417089F938F9388E292E09F938F93DF
:104C9000C3D70F900F900F900F90F80180819181F2
:104CA0000E9445136C01019609F4BACDD8011496FF
:104CB0008C911497823009F4DBC108F059C181301E
:104CC00009F0AECD8C2DF8019185923009F4BFC169
:104CD00008F075C1992309F47DC1913009F496C19A
:104CE000D80119961C929CCD68EFF80180819181C2
:104CF000D1DABFCF65EF8D919C91CCDA6AEEF801E5
:104D000080819181C7DABE016F5F7F4FC801FCDBF4
:104D100085E592E09F938F937FD768EED8018D91C0
:104D20009C91B8DA60E0F80180819181B3DA66EE97
:104D3000D8018D919C91AEDA66EEF8018081918167
:104D4000A9DA66EED8018D919C91A4DABE016F5F5D
:104D50007F4FC801D9DB0F900F908981882309F418
:104D600069C08A81882309F465C08EE492E09F932C
:104D70008F9352D766EEF801808191818BDA68EECD
:104D8000D8018D919C9186DA60E0F8018081918153
:104D900081DA68EED8018D919C917CDA63E0F801AC
:104DA0008081918177DA68EED8018D919C9172DAD9
:104DB00062E0F801808191816DDA68EED8018D9111
:104DC0009C9168DA61E0F8018081918163DA66EE96
:104DD000D8018D919C915EDA68EEF8018081918115
:104DE00059DA63E0D8018D919C9154DA68EEF801AC
:104DF000808191814FDA61E0D8018D919C914ADAEE
:104E000068EEF8018081918145DA62E0D8018D91E8
:104E10009C9140DA68EEF801808191813BDA63E091
:104E2000D8018D919C9136DA89E0F80184870F9042
:104E30000F9060C087E492E09F938F93EDD663EF6D
:104E4000D8018D919C9126DA68ECF80180819181DE
:104E500021DA63EFD8018D919C911CDA64E6F801A8
:104E60008081918117DA63EFD8018D919C9112DADC
:104E700060E5F801808191810DDAC8017BDB292F83
:104E800030E00F900F9083E02330310509F080E08F
:104E9000D8011C968C9380E492E09F938F93BCD6AC
:104EA00063EFF80180819181F5D968ECD8018D918B
:104EB0009C91F0D963EFF80180819181EBD968EC86
:104EC000D8018D919C91E6D963EFF80180819181A1
:104ED000E1D960E5D8018D919C91DCD9C8014ADB0C
:104EE000292F30E00F900F902430310529F584E010
:104EF000F801848764EFD8018D919C91CBD9BE01D4
:104F00006F5F7F4FC80100DBF8018485893021F194
:104F1000833029F1843031F1811127C08DE891E08F
:104F20009F938F938DE292E09F938F9375D60F900E
:104F30000F900F900F90A0CED8011C968C918111EC
:104F4000D9CF89E392E09F938F9366D666EFF801FD
:104F5000808191819FD96BCF83E791E0E1CF8CE78E
:104F600091E0DECF84E891E0DBCF85E991E0D8CF16
:104F7000833009F474C1843009F052CC8D919C9136
:104F800015D95C01019609F4BBC0D8018D919C91A3
:104F90000DD97C01019609F4B3C0F801848595858B
:104FA000853008F062C2833008F098C2882309F483
:104FB00095C240E0F12CE12CB12CA12CB6C393306A
:104FC00009F44EC0943009F08BCE65E5853C09F0BC
:104FD00087CE39C0813E51F08F3F09F478C0803EC2
:104FE00049F481E0D80119968C931ACC82E0F8013B
:104FF000818716CC6C2DC7FC04C0C8010E948510A7
:105000000FCC6F77C8010E945E100ACC863309F47A
:1050100067CE78F48A3209F463CE8C2DC7FC0FC0BA
:105020000E943511682FC8010E948510F801118671
:10503000F7CB8A3A09F454CE863B79F751CE8F7775
:105040000E943511682FC8010E945E10EFCF8D318C
:1050500029F08D3909F044CE84E0C9CF83E0C2CF76
:10506000853409F03DCE65E5C8010E94851038CE33
:10507000FC2C1A96EC911A97EB3008F063C0F0E024
:10508000EC5BF74D0C9405324F28B8289928E72897
:10509000FF2809290E29132919291E292929F80170
:1050A0008281938180599B4A029720F48C2D0E9423
:1050B000E406F82EF4E8FF16B9F1FF1558F020E8E1
:1050C000F21649F133E8F31641F1F1100DC00E94D8
:1050D000E614A6CB81EEF816D1F090EFF91691F018
:1050E000A0EE82E0FA16A1F06F2DF7FE86CF0E94A7
:1050F000AA108FEC91E09F938F938ED50F900F9015
:105100008CE0B8CB81E0D8011A968C9389CB84E0EF
:10511000F801828785CB89E0F6CF62E0C8010E9462
:105120008510F80112867CCB6FE7C8010E948510BC
:1051300009C0B9E5CB1631F0E0EFCE1639F0F2E157
:10514000CF1206C0D8011A961C926ACB83E0E0CF3A
:10515000D8011A961C92C7FC06C06C2DC8010E948B
:105160007B0F682F4ACF0E94AA1085EC91E0C3CF35
:10517000F8018281938180599B4A029720F48C2DFB
:105180000E94E406F82EF3E8FF16B9F024E8F216C0
:10519000C9F0D8011A961C926F2DF7FE33CF0E94EA
:1051A000AA101F92FF9286EB91E09F938F9334D5C4
:1051B0000F900F900F900F90A3CF62E0C8010E9454
:1051C0005E10C0CF6FE7C8010E945E10AACFB2E1A7
:1051D000CB1609F4B7CFE9E5CE1609F4B3CFD80161
:1051E0001A961C92C7FC06C06C2DC8010E947B0F4A
:1051F000682F08CF0E94AA1089EA91E07CCFB4E121
:10520000CB1629F0E0EFCE129DCF86E081CF85E06E
:105210007ACFF7E7CF1296CF60E087CFB4E1CB1219
:1052200091CF87E075CFF0EF88E0CF1609F46BCF10
:1052300089CFB7E7CB1286CF60E0C5CFF0EFCF12B2
:1052400002C08AE060CFF80112868C2D0E9482068F
:1052500088CF1A961C928C2D0E948206C9CF8C2D65
:105260008F3B29F090F496E59C0D923080F4D801A4
:105270001B961C9282EF91E09F938F93CDD48CE08C
:10528000F80180870F900F90CBCA8C3F81F3D80133
:105290001B969C911B97913009F473C098F0923043
:1052A00009F4BCC0933009F0BBCA8E3109F4DBC0ED
:1052B00008F0D0C061E5863109F0B8C0C8010E948D
:1052C0005E10C1C0F801228133812239FBEA3F0719
:1052D00019F58C3509F451C0B8F4833109F44FC085
:1052E000863809F43EC030F58338B9F1E0F48823FC
:1052F00009F4EDCE8038E9F187FF33CF85EE91E0F8
:105300009F938F9389D4BECF863721F08E3741F794
:1053100086E727CF8EE725CF21393B4A09F78C2D29
:105320000E940B07DDCF8438D1F068E6853809F498
:1053300064CEE2CF8C38C9F038F48738A1F061E050
:105340008B3809F45ACED8CF8D3889F0803FA1F63A
:1053500081E0D8011B968C9363CA62E04ECE6FE762
:105360004CCE68E74ACE60E048CE69E046CE6AE0BF
:1053700044CE82E0F801838753CA81E5F2CE8DE501
:10538000F0CE1B961C921B9712962D913C912239C0
:10539000BBEA3B0719F58C3509F437C0B8F4833103
:1053A00009F435C0EDE7E80FEB3098F5F0E0E55291
:1053B000F64D0C940532F529F729F929FB29FD2929
:1053C000092A092A092AFF29012A032A863721F0F6
:1053D0008E3741F786E70CCF8EE70ACF21393B4A5B
:1053E00009F78C2D0E940B07DDCF62E00BCE6FE733
:1053F00009CE68E607CE68E705CE60E003CE61E03F
:1054000001CE69E0FFCD6AE0FDCD81E5F1CE8DE50D
:10541000EFCE87FFEDCE8BED91E072CF8532B1F00C
:1054200040F48631A9F060E08E3151F00E94AA105C
:105430000AC0863221F0803FC9F783E08ACF6DE54C
:10544000C8010E948510F8011386EAC963E5F8CF08
:1054500061E5F6CF853229F06DE5863209F42ECF6D
:10546000E5CF63E52BCF60E029CF893009F0A1CDEE
:105470009601287433272834310509F037C1A1FE7D
:1054800035C1D594C794D594C794BCE0CB22DD2414
:10549000950154E0359527955A95E1F72370332708
:1054A0002C293D292230310509F4C7C023303105AC
:1054B00009F406C12130310509F028C1E6FC5CC0C1
:1054C0009701287033274E2D4F70E7FE39C080EFCB
:1054D000232B09F480E0482B80E038C0987F2C2DE6
:1054E0002770922BD8011D969C93C4FE02C0BB244A
:1054F000BA94C5FE02C0FF24FA94833009F40BC1AC
:10550000843009F0DBC0D8018D919C910E94D62097
:105510009C01019609F4D2C080EF23FF80E0422F66
:105520004F70842BF801958524FF01C19860958701
:10553000F801958525FFFEC09061958740E028C061
:1055400080EF232B09F480E0842B40E0E4FE16C0BA
:105550009860F8019587F80195855701F0E2AF2230
:10556000BB24E5FE10C09061D8011D969C93F12CE0
:10557000E12CB12CA12C0CC040E0AECF977FD8011C
:105580001D969C93E8CF9F7EF8019587F12CE12C26
:10559000F801958599832FE7F0E8AF16B10444F43C
:1055A000950191E8A9169FEFB90614F421E83FEFA1
:1055B0002A83A0E8EA16F1040CF0BFC0B1E8EB16AC
:1055C000BFEFFB0624F421E8E22EFF24FA94E194D5
:1055D000EB82803809F4B4C081958C83403809F49B
:1055E00041E84D83CE0101960E948509898180930F
:1055F0000D031F928F938D81282F082E000C330BE3
:105600003F938F938C81282F082E000C330B3F93F0
:105610008F938B81282F082E000C330B3F938F9391
:105620008A81282F082E000C330B3F938F9389E03B
:1056300092E09F938F93F0D2EECAE0FE2AC090646E
:105640009587D8011D968C911D97E1FE25C0806835
:105650001D968C93D8011D968C911D97E2FE20C05B
:1056600080621D968C93D8011D968C911D97E3FE48
:105670001BC080641D968C93D8011D968C91570198
:10568000B0E1AB22BB24E4FE13C08068F80185873B
:1056900090CC9F7B9587D5CF8F77F8018587DACF20
:1056A0008F7DF8018587DFCF8F7BF8018587E4CF79
:1056B0008F77D8011D968C93F12CE12C40E035C0FA
:1056C000A70134E0559547953A95E1F7842F8F70FF
:1056D00040E0E7FE03C0482F406F80E0987FBE2D7A
:1056E000B770EB2EE92AF801E58641CF987F8C2D23
:1056F0008770982BD8011D969C93C4FE02C0BB24D2
:10570000BA94C5FEDBCFFF24FA94D8CFF12CE12C5C
:10571000B12CA12CD3CFF801808191810E94D62099
:1057200040E08F3F980709F033CF80E031CF977F7B
:105730009587FECE9F7E958701CF91E8E92E48CFD1
:105740008FE74BCF0E9417089F938F9384E092E0DE
:105750009F938F9361D26EEFD8018D919C910E949F
:105760004A210F900F900F900F908A3A910511F4F3
:1057700089E080C80E9417089F938F938FEF91E074
:105780009F938F9349D2D80113961C921E92129721
:1057900014961C92149715961C920E94AA10F80158
:1057A000808191810E94DE100E94E614D801189633
:1057B0001C92ADC878941F920F920FB60F921124CD
:1057C0008F939F93AF93BF938091DD039091DE03FE
:1057D000A091DF03B091E0030196A11DB11D80935C
:1057E000DD039093DE03A093DF03B093E003BF914A
:1057F000AF919F918F910F900FBE0F901F901895B2
:105800001F920F920FB60F9211248F939F93AF9315
:10581000BF938091DD039091DE03A091DF03B091EF
:10582000E0034196A11DB11D8093DD039093DE033B
:10583000A093DF03B093E003BF91AF919F918F914D
:105840000F900FBE0F901F9018951F920F920FB6DA
:105850000F9211242F933F934F935F936F937F93F6
:105860008F939F93AF93BF93EF93FF938091E1004A
:1058700082FF09C08091E20082FF05C08091E100B3
:105880008B7F8093E1008091DA0080FF1FC08091C0
:10589000D80080FF1BC08091DA008E7F8093DA00F1
:1058A0008091D90080FFB9C080E189BD82E189BDC6
:1058B00009B400FEFDCF81E080930C038091DE02ED
:1058C000811104C00E94AD090E94E60D8091E100A3
:1058D00080FF21C08091E20080FF1DC08091E20026
:1058E0008E7F8093E2008091E20080618093E200ED
:1058F0008091D80080628093D80019BC85E08093A5
:105900000C038091E0028093DF021092E0020E947B
:10591000AA100E94A5148091E10084FF2FC08091FD
:10592000E20084FF2BC080E189BD82E189BD09B41A
:1059300000FEFDCF8091D8008F7D8093D8008091AC
:10594000E1008F7E8093E1008091E2008F7E809362
:10595000E2008091E20081608093E2008091030385
:10596000882309F460C084E080930C030E94AA108D
:105970000E94A5148091DF028093E0028091E100F3
:1059800083FF3AC08091E20083FF36C08091E1003E
:10599000877F8093E10082E080930C0310920303E1
:1059A0008091E1008E7F8093E1008091E2008E7F04
:1059B0008093E2008091E20080618093E20042E007
:1059C00060E080E00E94970A81E0809312011092CB
:1059D000E1031092E00280E2E1EEF2E0DF011D92CD
:1059E0008A95E9F7EBE9F2E01192B2E0EA3BFB07B6
:1059F000D9F781E080931001FF91EF91BF91AF91B2
:105A00009F918F917F916F915F914F913F912F91D6
:105A10000F900FBE0F901F90189519BC10920C0399
:105A20001092DE0253CF8091E30087FD02C081E037
:105A30009BCF83E099CF1F920F920FB60F92112444
:105A40002F933F934F935F936F937F938F939F9386
:105A5000AF93BF93EF93FF9384E094E00E94BF1F46
:105A6000FF91EF91BF91AF919F918F917F916F9136
:105A70005F914F913F912F910F900FBE0F901F900C
:105A800018951F920F920FB60F9211242F933F93E8
:105A90004F935F936F937F938F939F93AF93BF9336
:105AA000EF93FF9381E294E00E94BF1FFF91EF917B
:105AB000BF91AF919F918F917F916F915F914F9126
:105AC0003F912F910F900FBE0F901F901895FF934D
:105AD000EF93E0913E04F0913F04309709F009956F
:105AE000EF91FF910895FC018591803011F0EFDF77
:105AF000FBCF0895FF27E0E230E247FF0CC041955D
:105B000097FF09C0EDE26095709580959095611DB5
:105B1000711D811D911D27FF02C0219530E350E2C8
:105B2000AA27660F771F881F991FAA1FA41710F0B6
:105B3000A41B63955A95A9F7AA3008F0A95FA05D48
:105B4000AF93F395611571058105910541F7ED322C
:105B500011F4EF93F395F21718F43F93F395FBCFFD
:105B60008F91B5DFFA95E1F70895E991F991859163
:105B7000803021F0853219F0AADFF9CF089520E0B6
:105B8000E89455915532C1F3503311F4689455910E
:105B90005A3348F4505390F3220F022E220F220F53
:105BA000200D250FF4CF0EF421958991999153364C
:105BB00019F3533729F1533559F1BC018827992737
:105BC000E8945C3621F48991999168945591543602
:105BD00039F446EF7EF077FF0DC08FEF9FEF0AC0DC
:105BE00055374AE039F0583540E121F0523642E06D
:105BF00009F00895FF93EF937DDFEF91FF91B7CF09
:105C0000FF93EF93FC0181918030B9F360DFFBCF0C
:105C1000FF93EF9368DFF1CFDF93CF93CDB7DEB77C
:105C20002596A3DFCF91DF9108950F931F93CF9314
:105C3000DF93E6EFF3E001E214E0118300831382C7
:105C4000128214821582108611861286138614869B
:105C500015860E94AA10E8EEF3E0C4E0D4E0D183F8
:105C6000C0831382128214821582108611861286D6
:105C70001386148615860E94AA10F80111821082DC
:105C80001282138220E030E835832483168291E06B
:105C9000918F128E82E0838F948F198218821A82DC
:105CA0001B823D832C831E8293E0998F8A8F88E02C
:105CB0008B8F84E08C8FDF91CF911F910F9108958E
:105CC000CF93DF93CDB7DEB72A970FB6F894DEBF38
:105CD0000FBECDBF84B7877F84BF0FB6F894A89559
:105CE00080916000886180936000109260000FBE18
:105CF00080E890E00FB6F894809361009093610083
:105D00000FBE81E69EE090933F0480933E0486E0C0
:105D100091E09093D0038093CF038EEE94E0E3DE86
:105D20001092F9031092F8031092FA031092FB03F9
:105D30000E94AA108091F6039091F7030E94DE1052
:105D40001092EB031092EA031092EC031092ED0311
:105D50000E94AA108091E8039091E9030E94DE104E
:105D60000E94AD090E94E60D789482E084BD93E024
:105D700095BD9AEF97BD80936E008091E30381609B
:105D80008093E3030E94AA1080910C03843009F0F1
:105D90001AC10E94490E882309F415C18CED94E0C4
:105DA000A2DE8EEC94E09FDE80910C03853009F436
:105DB0000DC186EF93E00E942D2388EE93E00E94B0
:105DC0002D230CEC12E03BEB632E32E0732E512CB2
:105DD000F301A190B1903F01F801808091808A1475
:105DE0009B0409F460C08091E30381FF2EC08EEA1A
:105DF00094E079DE2BEBC22E22E0D22EF12CE12CA6
:105E0000F60180813180F2E0CF0ED11C0E94230880
:105E1000482E832D0E9423082AE431E03F932F93DC
:105E20004F928F93FF92EF9282EA94E09F938F9329
:105E3000F3DE8FEFE81AF80A0FB6F894DEBF0FBE54
:105E4000CDBFF8E0EF16F104D9F6D12CEE24E3949F
:105E5000F12CC4018A259B258E219F21892BE9F0F5
:105E6000DE825F8221E0C7018A219B21892B09F410
:105E700020E028870E9417088160782F9A878987F9
:105E80004E815F8168858A850E94391EF801808174
:105E900091818E259F2591838083D394EE0CFF1CE6
:105EA000F0E1DF12D6CF53940E5F1F4F88E05812F7
:105EB0008FCF8FEF89838A831B820E9417088160AE
:105EC000782F9D838C8349815A816B818D810E94BB
:105ED000391E8091D6039091D7030E940808AC0127
:105EE0009091D5032091170130E0911106C02091C7
:105EF0001801EAE02E9F900111244217530780F009
:105F00008091D9031091DA03F090DB030091DC0358
:105F1000811182C0111140C1F1103EC101113CC17B
:105F20000E94A1099091CB028917C1F00E94A1099A
:105F30008093CB029091E3039570953059F41F92B2
:105F40008F9383EC94E09F938F9366DE0F900F9076
:105F50000F900F908091CB020E9422232091E400A9
:105F60003091E5008091DC029091DD02281739071D
:105F700039F18091E4009091E5009093DD028093E7
:105F8000DC020E94490E8823D9F080910C038430F2
:105F9000B9F49091E9009F708091EC0080FFA4C05B
:105FA00080E8892B93E09093E9009091EB0090FFBB
:105FB00004C09091EE0097FDB5C08F708093E9000A
:105FC0000E94C90AF1CE0E94C90ADECE83B7817F42
:105FD0008C6083BF83B7816083BF7894889583B7D3
:105FE0008E7F83BF80910203882309F4DDCE86EF84
:105FF00093E00E942D2388EE93E00E942D23EBEB8B
:10600000F2E08BEC92E021913191232B09F0AEC0AC
:106010008E179F07C1F7C8CE9F3F19F09F5F9093DF
:10602000D503181624F40E94BE078093D9038091EB
:10603000D90387FF05C00E94BE0781958093D903CD
:10604000111624F40E94BE078093DA038091DA03CC
:1060500087FF05C00E94BE0781958093DA03609197
:10606000D903662301F11091DA031123E1F0062E22
:10607000000C770B880B990BC6D023E333E343E383
:106080005FE325D18DD06093D903612F110F770B7A
:10609000880B990BB8D023E333E343E35FE317D1D5
:1060A0007FD06093DA031F1424F40E948507809345
:1060B000DB038091DB0387FF05C00E948507819584
:1060C0008093DB03101624F40E9485078093DC0381
:1060D0008091DC0387FF05C00E948507819580932E
:1060E000DC030E94BD131CCF80E05BCFE091010177
:1060F000F0910201E90FF11D20819F5F30910501B0
:106100009323909304012093F1009091E80095FD72
:1061100009C09091E80090FF05C09091E8009E773B
:106120009093E8009091040120910301291721F038
:106130002091E80025FDDACF2091F3009091F20044
:10614000322F292F232B09F438CF9091E80090FFAC
:1061500034CF9091E80095FD06C09091E8009E77BD
:106160009093E8002ACF1092F100F3CF80E189BD2F
:1061700082E189BD09B400FEFDCF8091D8008F7DFA
:106180008093D8008091E00082608093E00080914D
:10619000E00081FDFCCF08CE9F3F09F03FCF50CFFC
:1061A00004D06894B1118DC0089570D088F09F57C5
:1061B00090F0B92F9927B751A0F0D1F0660F771F53
:1061C000881F991F1AF0BA95C9F712C0B13081F033
:1061D00077D0B1E0089574C0672F782F8827B85F13
:1061E00039F0B93FCCF3869577956795B395D9F794
:1061F0003EF490958095709561957F4F8F4F9F4F9E
:106200000895E89409C097FB3EF4909580957095A9
:1062100061957F4F8F4F9F4F9923A9F0F92F96E9F2
:10622000BB279395F695879577956795B795F11167
:10623000F8CFFAF4BB0F11F460FF1BC06F5F7F4F04
:106240008F4F9F4F16C0882311F096E911C0772316
:1062500021F09EE8872F762F05C0662371F096E81F
:10626000862F70E060E02AF09A95660F771F881FEE
:10627000DAF7880F9695879597F9089557FD905806
:10628000440F551F59F05F3F71F04795880F97FBFA
:10629000991F61F09F3F79F08795089512161306B4
:1062A0001406551FF2CF4695F1DF08C016161706E3
:1062B0001806991FF1CF8695710561050894089518
:1062C000E894BB2766277727CB0197F908950BD071
:1062D00078C069D028F06ED018F0952309F05AC024
:1062E0005FC01124EECFCADFA0F3959FD1F3950FC5
:1062F00050E0551F629FF001729FBB27F00DB11D4A
:10630000639FAA27F00DB11DAA1F649F6627B00DD9
:10631000A11D661F829F2227B00DA11D621F739FC2
:10632000B00DA11D621F839FA00D611D221F749FD0
:106330003327A00D611D231F849F600D211D822F17
:10634000762F6A2F11249F5750408AF0E1F088235E
:106350004AF0EE0FFF1FBB1F661F771F881F91506B
:106360005040A9F79E3F510570F014C0AACF5F3F7F
:10637000ECF3983EDCF3869577956795B795F7959E
:10638000E7959F5FC1F7FE2B880F911D9695879526
:1063900097F9089597F99F6780E870E060E00895A5
:1063A0009FEF80EC089500240A941616170618062D
:1063B0000906089500240A94121613061406050609
:1063C0000895092E0394000C11F4882352F0BB0F9A
:1063D00040F4BF2B11F460FF04C06F5F7F4F8F4FFD
:1063E0009F4F089597FB072E16F4009406D077FD73
:1063F00008D011D007FC05D03EF4909581959F4FB1
:106400000895709561957F4F0895EE0FFF1F0590D9
:10641000F491E02D0994AA1BBB1B51E107C0AA1FF0
:10642000BB1FA617B70710F0A61BB70B881F991F35
:106430005A95A9F780959095BC01CD010895F894DF
:02644000FFCF8C
:10644200059A010000FF460E6C1F3E1FFE1EC61E6F
:106452000101012808140A321E397F224D01CE00A3
:10646200AC00190532054B050102030405060708B5
:1064720009000008000400025F4E4F4E45005F45D0
:1064820052524F52005F5A313530005F49424D003F
:106492005F434C4F4E45005F49424D3834005854DB
:1064A200004154005445524D494E414C004D4F5508
:1064B2005345004C4F47495445434800494E5445C3
:1064C2004C4C49004558504C4F52455200444546A9
:0A64D20041554C54003F3F3F0000CD
:106800008800EA44E944E244040005000600070069
:10681000080009000A000B000C000D000E000F001C
:1068200010001100120013001400150016001700CC
:10683000180019001A001B001C001D001E001F007C
:10684000200021002200230024002500260027002C
:10685000280029002A002B002C002D002E002F00DC
:10686000300031003200330034003500360037008C
:10687000380039003A003B003C003D003E003F003C
:1068800040004100420043004400450046004700EC
:10689000480049004A004B004C004D004E004F009C
:1068A000500051005200530054005500560057004C
:1068B000580059005A005B005C005D005E005F00FC
:1068C0006000610062006300640065A185006700EC
:1068D000680069006A006B006C006D006E006F005C
:1068E0007000710072007300890087008A008B00BD
:1068F000E000E100E200E300E400E500E600E7007C
:106900000100010001000100EA4401000100E2442D
:106910000100010001000100460001004A004B0097
:10692000010001004700480001000100E9440100A6
:106930000100010001000100010001003A003B00DC
:106940003C003D003E003F0040004100420043004B
:10695000010035004C0039000100440045005200A0
:1069600049000100010050004F0029004D004E0079
:1069700051000100010001000100010001000100BF
:1069800001000100010001000100010001000100FF
:1069900001000100010001000100010001004D00A3
:1069A0004A004E004B0001000100010001000100FF
:1069B00001000100010001000100010001000100CF
:1069C00001000100010001000100010001000100BF
:1069D00001000100010001000100010001000100AF
:1069E0000100010001000100490001000100010057
:1069F000010001000100010001000100010001008F
:00000001FF
